:10079C002025322E58200025730020537973746560
:1007AC006D2048414C54454400204C6F632E20531F
:1007BC00746570706572206572726F720020537967
:1007CC007374656D20524553455400202E2E2E2EE9
:1007DC00204372656174696E672072616D702000D0
:1007EC00202E2E2E2E2E2046696E652061646A7591
:1007FC0073742020002044652D53796E6368726FEA
:10080C006E697A6564202000496E697420536C69A6
:10081C00646573202E2E2E002020202E2E2E20508C
:10082C006C65617365207761697400204D65636840
:10083C00616E6963616C204572726F7200202020BA
:10084C002E2E2E2053796E6368726F6E697A6564F2
:10085C00002E2E2E4F766572666C6F7720746F208B
:10086C004D494E2020002E2E2E556E646572666CFE
:10087C006F7720746F204D415820002E2E2E41642E
:10088C0076616E636520746F2025342E64002E2EE5
:10089C002E5265766572736520746F2025342E6434
:1008AC0000204D4F5645204572726F7200202E2E3F
:1008BC002E205361766500202E2E2E2045646974FF
:1008CC00002042617365202025332E64202D2030BA
:1008DC0078255820200020536C696465204E756D76
:1008EC0062657220256420002056616C75653A2083
:1008FC0025642073202000204379636C653A202501
:10090C0064207320200020456E61626C65642000B9
:10091C002044697361626C6564002056616C756576
:10092C003A202564205B25255D20200020466F722F
:10093C0077617264202000204261636B776172647E
:10094C007300204C4F4720202D202025322E640090
:10095C0020436F6E6669726D2052454C4F414420A6
:10096C002E2E2E00202E2E2E204C6F6164656400DE
:10097C002045726173652043616C696272617469B0
:10098C006F6E203F00202E2E2E2045726173656401
:10099C00002041646A75737420506F736974696FB9
:1009AC006E0020536C6964652025322E64204465EA
:1009BC00762025322E642000205361766520536505
:1009CC007474696E6773202E2E2E20200020436FC6
:1009DC006E6669726D20434D44202E2E2E002053DE
:1009EC00656C65637420536C69646520312021212A
:1009FC00002056616C75653A202564205B312F31DF
:100A0C0030206D6D5D20200020436F6E6669726D25
:100A1C002054657374202E2E2E00205344785020C1
:100A2C00434F4D4D206572726F72200020534478F5
:100A3C005020434F4D4D2070617373656400204D01
:100A4C004F56454D454E54207061737365642000BC
:100A5C00204D4F56454D454E54206572726F722095
:100A6C002000204465766963652046554E43544901
:100A7C004F4E204F4B202000204465766963652043
:100A8C004D414C46554E4354494F4E202000536F18
:100A9C006674205265736574202E2E2E00202E2E27
:100AAC002E20506C65617365205761697400202E8F
:100ABC002E2E2053656C656374202020202020206E
:100ACC00202000202E2E2E2045646974202000202A
:100ADC002E2E2E2043616E63656C20496E707574EA
:100AEC0000202E2E2E2053656C65637400534C49E8
:100AFC00444520564945572020434F4D50202F3117
:100B0C00320076657273696F6E20322E3538005064
:100B1C004547415355532039382E2E2E3031002065
:100B2C005344785020434F4D4D206572726F7200C4
:100B3C00494E495420627970617373656400257362
:100B4C00202D2025322E64202F2025322E642000CB
:100B5C002054696D65206C6566743A2025332E64CB
:100B6C00202020200020416E616C6F67205B2525C2
:100B7C005D2025322E642025322E64202000204159
:100B8C0075746F205363726F6C6C696E67002044D0
:100B9C006D782025332E64202D2025332E642025BE
:100BAC00332E64202000000000000000090000002B
:100BBC0011FF00001AFF000023FE00002CFE0000B5
:100BCC0035FD00003EFD000047FC000050FC00001D
:100BDC0059FB000062FB00006BFA205072696D61DA
:100BEC00727920636F6E74726F6C2020000020533A
:100BFC00657175656E7469616C206163636573738F
:100C0C0000002052616E646F6D20416363657373E5
:100C1C00202020200000204175746F2054696D65E0
:100C2C0072202020202020200000205363726F6C43
:100C3C006C696E672020202020202020000020538B
:100C4C00696E676C65202020202020202020000069
:100C5C0020556E692D446972656374202020202014
:100C6C0000002042692D44697265637420202020A5
:100C7C002020000020556E692D4469726563742034
:100C8C00496E742E00002042692D446972656374AC
:100C9C0020496E742E2000004F7065726174696F6C
:100CAC006E206D6F646520200000444D58206164F7
:100CBC00647265737320202020200000536C6964DB
:100CCC0065204E756D6265722020202000004578ED
:100CDC00706F737572652074696D6520202000003B
:100CEC00466164696E672074696D65202020202040
:100CFC0000004175746F54696D6572204D6F6465A9
:100D0C00202000005368757474657220436F6E74F4
:100D1C00726F6C2000005363726F6C6C2073706583
:100D2C0065642020202000005363726F6C6C20647B
:100D3C006972656374696F6E000041636F757374DB
:100D4C0069632062656570202020000052656C6F1D
:100D5C0061642064656661756C7473200000436186
:100D6C006C6962726174696F6E2020202020000013
:100D7C0042656C7420636F7272656374696F6E2068
:100D8C0000004572726F7220636F64652020202012
:100D9C0020200000446961676E6F7374696373206F
:100DAC002020200000005072696D61727920005380
:100DBC00657175656E63650052616E646F6D2020A0
:100DCC000054696D6572202020005363726F6C6C47
:100DDC0020200020204E6F20726563657074696F4F
:100DEC006E004E6F2044494D4D4552206461746134
:100DFC0000202020446D782064617461204F4B00EA
:100E0C0013202D394653606C7986939FACB9C6D2AA
:1032CB00C113C115C114C192C116C111C11701623D
:0132DB0000F2
:05333200D2F8D2F922DF
:082699008F408B418A42894306
:1026A100C2F8120048C2F9E54025E054FEF540E4C5
:1026B100FFE54025E0F54092F8D2F9C2F90FBF08D5
:1026C100F0D2F8D2F9A2F8B3920AC2F9200902D2E3
:1026D1000A300A41E544603DAB41AA42A9431212C6
:1026E1006EFEE4FFEE25E0FE92F8D2F9C2F90FBFCB
:1026F10008F2D2F8D2F9A2F8B3920AC2F97401250C
:1027010043F543E43542F5421544200902D20AD289
:10271100AED2BE80BCC2F8D2F9120048D2F8A20AE9
:012721002295
:0820E5008F3F8B408A418942C4
:1020ED00E4F545754680C2F8120048C2F9E53F2572
:1020FD00E04401F53FE4F544E53F25E0F53F92F876
:10210D00D2F9C2F90544E544B408EDD2F8D2F9A2EA
:10211D00F8B39208C2F9300850E543604CE4FFF57E
:10212D0044D2F930F804E5464207C2F9E546C31337
:10213D00F5460544E544B408E8AB40AA41A942EF91
:10214D001212871543E5436004C2F88002D2F8D21B
:10215D00F9120048C2F974012542F542E43541F502
:10216D00410545D2AED2BE80ADC2F8D2F9120048BB
:04217D00D2F8AF45A0
:01218100223B
:10310E00C208753F0A786AA60708A60520081FE5BB
:10311E003F601B7F017E001200037B007A00796AFC
:10312E00754402D2097F50122699920880DEA208B9
:01313E00226E
:10303500C205752E0A786AA607ECFF3395E0EF08FE
:10304500F6ED08F620051FE52E601B7F017E0012B8
:1030550000037B007A00796A754403D2097F501218
:083065002699920580DEA20508
:01306D002240
:1031C400786AA6077B007A00796A754401D2097F80
:1031D400501226997B007A00796A7543017F501258
:0731E40020E5786AE6FF22F6
:022D6B008F37A0
:102D6D00786AA6377B007A00796A754401D2097FAB
:102D7D00501226997B007A00796A7543017F5012B3
:102D8D0020E5786AE6F538E53704F67B007A0079B8
:102D9D006A754401D2097F501226997B007A007919
:102DAD006A7543017F501220E5E538FE786AE67CAE
:072DBD00002400FFEC3EFEC4
:012DC40022EC
:05333700D2B4D2B52262
:042EB2008F3A8D3B8B
:102EB600E53B6030A83AE6F53D753C08E53C601711
:102EC600E53D25E0F53D153C92B4C2B5D2B57F642B
:102ED6007E0012316F80E5053A153B7F647E001255
:102EE600316F80CCD2B4D2B57FF47E0112316F300F
:052EF600B402C322D369
:012EFB0022B4
:102E6700752F7820940BA20692087F0A7E001230F5
:102E77006E43E80FD2EED2ECE5E8540FF52E30059D
:102E87001D20941AE52F600B7F0A7E0012000315A0
:102E97002F80EED2087F0A7E0012306E80E3C2EEEA
:0A2EA700C2ECC2C1C213D2B9AF2EB3
:012EB10022FE
:1031EB00752B7820941AE52B600B7F0A7E0012005A
:1031FB0003152B80EED2087F0A7E0012306E80E31F
:06320B00C2C1C213D2B9DA
:01321100229A
:0D330D003094097F017E0012000380F4223D
:022EFC008F3C09
:102EFE007F301231C48F3DE53D2431FFAD3C1231A0
:102F0E000E053DE53DC3940550028001C34003E428
:102F1E00F53DAD3D7F3012310EE4F53ED2087F1EF9
:102F2E007E0012306E7FC87E00120003053EE53E25
:052F3E00C3940640E70A
:012F4300226B
:102DC5007F301231C48F2C152CE4F52DE52CC394DE
:102DD5000550028001C34003752C04E52C2431FF06
:102DE5001231C4742E252DF8A607152C052DE52DB9
:102DF500C3940540D7E4F52D7BFF7A07799C742EA3
:102E0500252DF8E6753F00F540120E7E052DE52DC2
:052E1500C3940540E339
:012E1A002295
:10323800E4FD7F3012310EE4F52CE52C2431FF7DBE
:0D324800FF12310E052CE52CC3940540ED5E
:013255002256
:102FC1008B2C8A2D892E12328D7F401232B8852C9E
:102FD1003F852D40852E417BFF7A0779A3120E7E16
:102FE1007F141232B87BFF7A0779A6120E7E7FF228
:0A2FF100122EFCD2AED2BE80FA22EE
:10313F0012328D7F401232B87BFF7A0779B5120EAB
:10314F007E7F141232B87BFF7A0779C9120E7E7F09
:10315F00F1122EFCD2087FD07E0712306E80FE2235
:042722008F2D8D2E3C
:10272600752F05753005C204786A768008768108AB
:102736007682796AE718262482786DF6200445E5C4
:10274600306041E52DC313452EFF7B007A00796A80
:10275600754404D2091226994011E52F600DD2085E
:102766007F0A7E0012306E152F80D87F907E011270
:10277600316F20F904D20480077F327E00120003F5
:10278600153080B87FC87E00120003E52F6006E58D
:10279600306002D322D2087FD07E0712306E12310B
:0227A6003FC32F
:0127A800220E
:082346008F348D358A368B3788
:10234E00753805753905C204786A7690E536FF331F
:10235E0095E0EF08F6AF37E53708F6FF796AE7182C
:10236E00262F786DF6200445E5396041E534C31318
:10237E004535FF7B007A00796A754404D20912262E
:10238E00994011E538600DD2087F0A7E0012306E3A
:10239E00153880D87F907E0112316F20F904D20457
:1023AE0080077F327E00120003153980B87FC87E09
:1023BE0000120003E5386009E5396005AE36AF3727
:0823CE002212313F7EFF7FFF68
:0123D60022E4
:042A35008F2F8D3022
:102A3900753305753405C205786A76A008A60308BA
:102A4900A632796AE718262532786DF6200545E51C
:102A5900346041E52FC3134530FF7B007A00796A62
:102A6900754404D2091226994011E533600DD20844
:102A79007F0A7E0012306E153380D87F907E011256
:102A8900316F20F904D20580077F327E00120003DE
:102A9900153480B87F647E00120003E5336006E5D3
:092AA900346002D32212313FC354
:012AB2002201
:04221C008F2A8D2B4D
:10222000753005753105C203786A76C0AE02AF031A
:102230007C007D64121300786BA607AE2EAF2F7C56
:10224000007D64121300786CEFF6796AE718262F88
:10225000786DF6200345E5316041E52AC313452B2F
:10226000FF7B007A00796A754404D20912269940EE
:1022700011E530600DD2087F0A7E0012306E1530F5
:1022800080D87F907E0112316F20F904D20380073D
:102290007F327E00120003153180B87F647E001209
:1022A0000003E5306006E5316002D32212313FC3FE
:0122B000220B
:0428B3008F2A8D2BB0
:1028B700752F05753005C203786A76B008A603E55B
:1028C7002DC313E52E13FF08F6796AE718262F782C
:1028D7006DF6200345E5306041E52AC313452BFF1C
:1028E7007B007A00796A754404D20912269940114F
:1028F700E52F600DD2087F0A7E0012306E152F80FB
:10290700D87F907E0112316F20F904D20380077FB0
:10291700327E00120003153080B87F647E001200FB
:0F29270003E52F6006E5306002D32212313FC373
:01293600227E
:042AB3008F2A8D2BAE
:102AB700752E05752F05C203786A76D008A6030818
:102AC700A62D796AE71826252D786DF6200345E5AA
:102AD7002F6041E52AC313452BFF7B007A00796AF3
:102AE700754404D2091226994011E52E600DD208CB
:102AF7007F0A7E0012306E152E80D87F907E0112DD
:102B0700316F20F904D20380077F327E0012000361
:102B1700152F80B87F647E00120003E52E6006E55E
:092B27002F6002D32212313FC3DA
:012B30002282
:042937008F2A8D2B2B
:10293B00752C05752D05C203786A76E0EA08F6AFAB
:10294B0003EB08F6796AE718262F786DF620034516
:10295B00E52D6041E52AC313452BFF7B007A0079F7
:10296B006A754404D2091226994011E52C600DD2E8
:10297B00087F0A7E0012306E152C80D87F907E0166
:10298B0012316F20F904D20380077F327E001200D0
:10299B0003152D80B87F647E00120003E52C6006C2
:0A29AB00E52D6002D32212313FC374
:0129B50022FF
:0429B6008F2F8D30A2
:1029BA00753105753205C205786A7620300404E659
:1029CA004401F6786B76AA0876BB796AE71826245A
:1029DA00BB786DF6200545E5326041E52FC3134506
:1029EA0030FF7B007A00796A754404D2091226996D
:1029FA004011E531600DD2087F0A7E0012306E1553
:102A0A003180D87F907E0112316F20F904D205807F
:102A1A00077F327E00120003153280B8E531600666
:0A2A2A00E5326002D32212313FC3EF
:012A3400227F
:082467008F348D358A368B3766
:10246F00753A05753B05C205D3E5379539E53695C0
:10247F00384006853836853937786A7638E5360834
:10248F00F6AF37E53708F6FF796AE718262F786D2C
:10249F00F6200545E53B6041E534C3134535FF7B29
:1024AF00007A00796A754404D2091226994011E521
:1024BF003A600DD2087F0A7E0012306E153A80D82E
:1024CF007F907E0112316F20F904D20580077F3291
:1024DF007E00120003153B80B8E53B6005AE36AFBA
:0524EF00372212313F0D
:0124F40022C5
:0419D2008F2E8D2F98
:1019D600753605753705C207E5332BE5323AC394EC
:1019E600005009C3E49BF533E49AF532E5332BFF47
:1019F600E5323AFED3EF9535EE9534400AE5359B50
:101A0600F533E5349AF532D3E5339400E532648054
:101A160094804008786A7611D2068006786A761035
:101A2600C206300506786AE64404F6AF33AE3212D3
:101A360032DD8E328F33E53345327003021AC8E544
:101A460032FF3395E0EF786BF6AF33E53308F6FFF8
:101A5600796AE718262F786DF6200745E537604145
:101A6600E52EC313452FFF7B007A00796A7544047F
:101A7600D2091226994011E536600DD2087F0A7EFA
:101A86000012306E153680D87F907E0112316F209D
:101A9600F904D20780077F327E00120003153780D3
:101AA600B8E53760197F037E00120003300605AEE5
:101AB60032AF3322C3E49533FFE49532FE2212316E
:061AC6003F227E007F00BC
:011ACC0022F7
:10189000300450AD5FAC5E7F10123035AD5B7F23FE
:1018A00012310EAD547F2012310EAD557F2412310E
:1018B0000EAD567F2512310EAD577F2212310EAD7F
:1018C0005C7F2612310EAD587F2712310EAD5D7F41
:1018D0002912310EAD5A7F2812310EAD597F2112D7
:1018E000310E227F10122D6B8E5E8F5FC3E55F94E9
:1018F00001E55E9400400BD3E55F94FCE55E940146
:101900004006755E00755F017F231231C48F5BD383
:10191000E55B648094845009C3E55B6480948050E7
:1019200003E4F55B7F201231C48F54E554D3940C4B
:101930005007E554C39401500375540C7F241231B1
:10194000C48F55E555D394965007E555C39401507F
:101950000375550A7F251231C48F56E556D3943C42
:101960005007E556C3940150037556057F26123182
:10197000C48F5CD3E55C648094855009C3E55C64E6
:101980008094815003755C027F271231C48F58E523
:1019900058D394645007E558C394015003755850C8
:1019A0007F291231C48F5DD3E55D6480948A50092C
:1019B000C3E55D648094765003E4F55D7F281231C1
:1019C000C48F5A7F211231C48F597F221231C48FA4
:0219D00057229C
:0B33270075988075A910C298C2992209
:1030A60053D8F8EF540742D8C2DBE4F52A75DA8024
:1030B60020DCFD746A252AF8A6D97F037E0012005B
:1030C60003052AE52AC3940340E37F6A7D03122F92
:0530D600FB786BE6FF32
:0130DB0022D2
:10327200D291EF25E054074401786AF608A6057F4B
:0B3282006A7D02122EB2C291D291228E
:041D77008F348D35E3
:101D7B007F541232B87BFF7A0779D7120E7EE53487
:101D8B00601FFF3395E0FE7C007D0E1212997C6381
:101D9B007D9CCFCDCFCECCCE1213008E368F37801D
:101DAB000675366375379CE535249B604D046003DF
:101DBB00021E4CE4F538F539AE38AF397C007D6442
:101DCB00121300AD07E4FF1232727F477E00120040
:101DDB0003E5372539F539E5363538F538C3E539B7
:101DEB00949CE538648094E340CE7DFFE4FF12328F
:101DFB00727D147F041230DCC32275386375399CF5
:101E0B00AE38AF397C007D64121300AD07E4FF12CE
:101E1B0032727F477E00120003C3E5399537F539DF
:101E2B00E5389536F538D3E5399400E53864809478
:101E3B008050CDE4FDFF1232727D147F041230DC32
:011E4B00D3C3
:011E4C002273
:101C9D007F541232B87BFF7A0779EC120E7E7532C3
:101CAD003CE4FBFD7FB0122A3530B229C204E4FDBD
:101CBD007FB01229B6752D4E752E2030B217E52E38
:101CCD00452D60117F017E00120003E52E152E704B
:101CDD0002152D80E6D204E4FD7FB01229B6752DD4
:101CED004E752E2020B217E52E452D60117F017EF9
:101CFD0000120003E52E152E7002152D80E6C2F898
:101D0D007F017E00120003D2F87F647E0012000373
:101D1D0075386C7539BC7B037A00E4FD7FB01224F5
:101D2D00677FFA7E00120003E55825E02419F5328D
:101D3D00E4FBFD7FB0122A35D2127B057A00E4FD5B
:101D4D007FB0122346C211E52E452D70157F54121A
:101D5D0032B87BFF7A087901120E7E7F12122EFCAB
:091D6D0080FE7D147F041230DCBD
:011D7600224A
:102F44007532A0E4FBFD7FB0122A35752D00752E75
:102F5400FA7B24E4FD7FB01228B3752E05752F1477
:102F64007B587A02E4FD7FB012221CE4F52D7B64C9
:102F7400FD7FB0122AB37B587A6CE4FD7FB012292E
:022F84003722F2
:10260E007BFF7A087914120E7E7F401232B87BFF60
:10261E007A087924120E7E20B25A7B587A6CE4FD29
:10262E007FB0122346C204E4FD7FB01229B67FE8C4
:10263E007E03120003752A4E752B2020B217E52B50
:10264E00452A60117F057E00120003E52B152B70C5
:10265E0002152A80E6C2F87F017E00120003D2F82E
:10266E00E52B452A700E7F10122EFC7BFF7A08791F
:10267E0037122FC17F141232B87BFF7A08794912B4
:0A268E000E7E121C9D12328D7F019A
:01269800221F
:022182008F3498
:102184001534E534700302221725E02440FF122D94
:102194006B8E358F36E53425E025E024B2F582E4F4
:1021A400340BF583121347EF241EFBE43EFAE43D9F
:1021B400F9E43CF8AE35AF36E4FCFDC31213364007
:1021C4002FE53425E025E024B2F582E4340BF583D1
:1021D400121347EF24E2FBEE34FFFAED34FFF9EC7F
:1021E40034FFF8AE35AF36E4FCFDD3121336401E8F
:1021F4007D037C007FC87E00122046E53425E0255F
:10220400E024B2F582E4340BF58312134722AE3591
:07221400AF36227E007F00BF
:01221B0022A0
:0613E6008F2D8C2E8D2FCF
:1013EC00852D30753105E562B52D01227F14123241
:1013FC00B8E52F452E600DE55760097D65AF561297
:10140C001D779217E52DB4011AE554C3132401FF7F
:10141C00E433FED3E5629FEE6480F8748098400359
:10142C00752D0D75310520FF0302157BE52DD39528
:10143C0054405C7BFF7A08795D120E7E3012277F58
:10144C000D122182AD5DED3395E0FCEF2DFFEE3CEE
:10145C00CF2405FBE43FFA75386C7539BCE4FD7F8D
:10146C00B0122467801F7F0D122182AD5DED339584
:10147C00E0FCEF2DFBEE3CFA75386C7539BCE4FDE5
:10148C007FB0122467B211D21275300102156BE5D0
:10149C002DC3940150673012157F0D122182EF2459
:1014AC0005FBE43EFAE4FD7FB012234680107F0D6D
:1014BC00122182AA06AB07E4FD7FB01223467BFF04
:1014CC007A087972120E7EE55BB4030FE55CB40406
:1014DC000AE55420E00514F52D800385542DAF2D1D
:1014EC00122182AA06AB0775386C753958E4FD7F5A
:1014FC00B0122467B211C212852D308062E52DD353
:10150C0095624030AF2D1221828E328F33EF24053D
:10151C00FBE43EFA75386C753958E4FD7FB0122443
:10152C0067D2127BFF7A08798785323F8533401268
:10153C000E7E802BAF2D122182AA068A32AB078B2E
:10154C003375386C753958E4FD7FB0122467C212BC
:10155C007BFF7A08799A85323F853340120E7E7F65
:10156C00647E001200031531E5316003021432E58C
:10157C003170157F541232B87BFF7A0879AD120E98
:0C158C007E7F11122EFC80FED216AF30C4
:011598002230
:03004B0002333C41
:05333C00D213C2B932FA
:03002300022C9F0D
:102C9F00C0E0C0D075D008309A41301556301418A6
:102CAF00C214E59960057563018048756302E5619B
:102CBF00156170021560803BE5614560600AE56152
:102CCF00156170021560802B74652564F8A699E56F
:102CDF006460041564801CC2158018E599700F8517
:102CEF005E60855F61756404D214D2158005C215CC
:0A2CFF0075630AC298D0D0D0E0320D
:101E4D00855B2BC203D205A2039206122E67EF64A7
:101E5D0002607BBF040E155BC3E55B64809480500C
:101E6D0003E4F55BBF080E055BD3E55B64809484EA
:101E7D004003755B04EF640170287F541232B87B08
:101E8D00FF7A0879B9120E7ED2041218907FE87E7F
:101E9D00031200037F541232B87BFF7A0879C31204
:101EAD000E7E7F401232B8AF5BEF3395E0FE7C00C3
:101EBD007D1412129974E62FF9740B3EFA7BFF1202
:101ECD000E7EE55924FF920312330D021E52E52BAF
:101EDD00B40408E55B6404600280FEE52B640360D6
:101EED0010E55BB4030B7D017C007F011213E68FBF
:011EFD006282
:011EFE0022C1
:101EFF00C205C206122E67EF64027003021F98BF5D
:101F0F000417055FE55F7002055ED394FCE55E94F0
:101F1F00014006755E00755F01BF0819E55F155F2B
:101F2F007002155EC3E55F9401E55E94005006757F
:101F3F005E01755FFCEF640170287F541232B87B2D
:101F4F00FF7A0879B9120E7ED2041218907FE87EBC
:101F5F00031200037F541232B87BFF7A0879C31241
:101F6F000E7E7F401232B87BFF7A0879CD855E3FB7
:101F7F00855F40855E41855F42120E7E7FC87E0081
:101F8F0012000312330D021EFFE55924FF92087F42
:061F9F000A7E0012306E04
:011FA5002219
:1023D70085542BC205C206122E67EF6402606BBFDD
:1023E700040C0554E554D3940C400375540CBF08F2
:1023F7000C1554E554C394015003755401EF64015F
:1024070070287F541232B87BFF7A0879B9120E7E92
:10241700D2041218907FE87E031200037F54123211
:10242700B87BFF7A0879C3120E7E7F401232B87BE1
:10243700FF7A0879E2753F00855440120E7E7FC807
:102447007E0012000312330D8089E55924FF92089C
:0F2457007F0A7E0012306EE554652B600280FE16
:012466002253
:1027A900C205C206122E67EF6402606BBF040C05F6
:1027B90055E555D394964003755501BF080C155539
:1027C900E555C394015003755596EF640170287F50
:1027D900541232B87BFF7A0879B9120E7ED20412EC
:1027E90018907FE87E031200037F541232B87BFFF2
:1027F9007A0879C3120E7E7F401232B87BFF7A08BD
:1028090079F4753F00855540120E7E7FC87E00120F
:10281900000312330D8089E55924FF92087F0A7E4F
:042829000012306EFB
:01282D002288
:10282E00C205C206122E67EF6402606BBF040C0570
:10283E0056E556D3943C4003755601BF080C155609
:10284E00E556C39401500375563CEF640170287F22
:10285E00541232B87BFF7A0879B9120E7ED2041266
:10286E0018907FE87E031200037F541232B87BFF6C
:10287E007A0879C3120E7E7F401232B87BFF7A0936
:10288E007903753F00855640120E7E7FC87E00127A
:10289E00000312330D8089E55924FF92087F0A7ECA
:0428AE000012306E76
:0128B2002203
:102B3100C203D205A2039206122E67EF64026069F6
:102B4100EF64046003BF080CE55770047E01800246
:102B51007E008E57EF640170287F541232B87BFFDC
:102B61007A0879B9120E7ED2041218907FE87E039A
:102B71001200037F541232B87BFF7A0879C3120E18
:102B81007E7F401232B8E557600B7BFF7A097912DC
:102B9100120E7E80097BFF7A09791C120E7EE5599F
:092BA10024FF920312330D808918
:012BAA002208
:101FA600855C2BC203D205A2039206122E67EF644C
:101FB60002607BBF040E155CC3E55C6480948150AF
:101FC60003755C01BF080E055CD3E55C64809485EF
:101FD6004003755C05EF640170287F541232B87BAC
:101FE600FF7A0879B9120E7ED2041218907FE87E25
:101FF600031200037F541232B87BFF7A0879C312AA
:102006000E7E7F401232B8AF5CEF3395E0FE7C0067
:102016007D1212129974382FF9740C3EFA7BFF1256
:102026000E7EE55924FF920312330D021FABE52BFA
:0F203600655C600B7D017C007F011213E68F62F9
:012045002278
:1022B100C205C206122E67EF6402606BBF040C05F3
:1022C10058E558D394644003755801BF080C15585C
:1022D100E558C394015003755864EF640170287F79
:1022E100541232B87BFF7A0879B9120E7ED20412E9
:1022F10018907FE87E031200037F541232B87BFFEF
:102301007A0879C3120E7E7F401232B87BFF7A09B8
:102311007926753F00855840120E7E7FC87E0012D7
:10232100000312330D8089E55825E02419F532E4C4
:10233100FBFD7FB0122A35E55924FF92087F0A7E02
:042341000012306EE8
:012345002275
:102BAB00C203D205A2039206122E67EF640260697C
:102BBB00EF64046003BF080CE55A70047E018002C9
:102BCB007E008E5AEF640170287F541232B87BFF5F
:102BDB007A0879B9120E7ED2041218907FE87E0320
:102BEB001200037F541232B87BFF7A0879C3120E9E
:102BFB007E7F401232B8E55A600B7BFF7A09793839
:102C0B00120E7E80097BFF7A097943120E7EE559FD
:092C1B0024FF920312330D80899D
:012C2400228D
:102E1B00C2037D147F041230DCD205A2039206128A
:102E2B002E678F2BEF6402602B7F401232B87F30FE
:102E3B001231C4753F008F407BFF7A09794E120E19
:102E4B007E7F141232B8122DC5E55924FF9203125E
:0B2E5B00330D80C57D147F031230DCB6
:012E66002249
:102C2500C203D205A2039206122E67EF6402606901
:102C3500EF64046003BF080CE55970047E0180024F
:102C45007E008E59EF640170287F541232B87BFFE5
:102C55007A0879B9120E7ED2041218907FE87E03A5
:102C65001200037F541232B87BFF7A0879C3120E23
:102C75007E7F401232B8E559600B7BFF7A097912E5
:102C8500120E7E80097BFF7A09791C120E7EE559AA
:092C950024FF920312330D808923
:012C9E002213
:101ACD00C2037F401232B87BFF7A09795C120E7E19
:101ADD00E55924FF920312330DD205A2039206128B
:101AED002E67EF64016003021BB8F55BF55E755F51
:101AFD000175540C75550A755605F557755C0275CB
:101B0D005850755A017559011232387F541232B836
:101B1D007BFF7A097970120E7ED2041218907FE83D
:101B2D007E031200037D147F041230DC7F401232DD
:101B3D00B87BFF7A09797C120E7E12330DD205A285
:101B4D00039206122E67EF64017060F52BD3E52B1F
:101B5D006480948C4003D38001C34033E52B25E092
:101B6D002440FFC007AF2BEF3395E0FEEF7802C3A3
:101B7D0033CE33CED8F924B2F582740B3EF58312F1
:101B8D001347AD07AC06D007123035052B80BE7F4D
:101B9D00541232B87BFF7A097991120E7E7FE87E5E
:0B1BAD00031200037D147F041230DCE3
:011BB800220A
:10159900C203C204E56264016003021715D205A201
:1015A900039206122E678F2BEF6402700302172A2B
:1015B900E562640C700302172AE52B6401600302DB
:1015C90016FB7F401232B87BFF7A09799D120E7E95
:1015D900755850E55825E02419F532E4FBFD7FB034
:1015E900122A35756202E562D3940C4003D3800157
:1015F900C350030216F9E56225E025E024AEF58221
:10160900E4340BF583121347EF24E7FBEE34FFFABA
:1016190075386C753958E4FD7FB01224677FFA7EFE
:1016290000120003752DC220FF0A7F327E001200CE
:1016390003D52DF3E52D700280FE752CE27F54123F
:1016490032B87BFF7A0979AE753F00856240AF2CCD
:10165900EF3395E0F5418F42120E7E12330DD2051C
:10166900A2039206122E678F2BE52B6404702D05B9
:101679002CF53275330175346C753558C205FBFA92
:10168900FD7FB01219D2752DC220FF0A7F0A7E0094
:10169900120003D52DF3E52D700280FEC3E52C64FD
:1016A90080949E5006E52B640170927F541232B8E3
:1016B9007BFF7A0979C4120E7EE56225E025E024D4
:1016C900AEF582E4340BF583121347AD2CED339557
:1016D900E0FCEF2DFDEE3CFCE56214FF25E0244023
:1016E900FF1230357FE87E0312000305620215EF11
:1016F90080FE7F401232B87BFF7A0979D9120E7EBB
:10170900E55924FF920312330D0215A67F401232C8
:10171900B87BFF7A0979EA120E7E7FE87E03120010
:0117290003BC
:01172A00229C
:1024F500C205C206122E67EF64026073BF040E05A3
:102505005DD3E55D6480948A4003755D0ABF080E5E
:10251500155DC3E55D648094765003755DF6EF64E3
:102525000170287F541232B87BFF7A0879B9120EF0
:102535007ED2041218907FE87E031200037F5412A6
:1025450032B87BFF7A0879C3120E7E7F401232B80B
:102555007BFF7A0979FDAF5DEF3395E0F53F8F405D
:10256500120E7E7FC87E0012000312330D8081E5B6
:0C2575005924FF92087F0A7E0012306E8D
:012581002237
:101BB900C2037F401232B87BFF7A0A7914120E7E73
:101BC90012330DD205D206122E67EF6401600302AB
:101BD9001C9C7F401232B8E4FD7FB0122722400DD1
:101BE9007BFF7A0A7926120E7ED20380097BFF7A5F
:101BF9000A7938120E7E7FD07E071200037532A053
:101C0900E4FBFD7FB0122A35E4FDFC7F011213E6E7
:101C19008F627FDC7E05120003752B0B752CB820B3
:101C2900FF1A7F0A7E00120003E52C152C7002159D
:101C39002BD3E52C9400E52B940050E37D147F030E
:101C49001230DC7F401232B8E52C452B600B7BFF4C
:101C59007A0A794A120E7E800B7BFF7A0A795C1226
:101C69000E7ED2037FD07E0712000320030E121CC2
:101C79009D7BFF7A0A796E120E7E80097BFF7A0AB4
:101C89007984120E7E7F401232B87F887E1312004B
:031C99000380FEC7
:011C9C002225
:10319A0012328DE4FF1232B87BFF7A0A799A120E44
:1031AA007E7F401232B87BFF7A0A79A9120E7E120C
:0A31BA0031EB7FF0122EFC80FE22A4
:10172B00E4F52A12328DE4FF1232B8AF2AEF33956B
:10173B00E0FE7C007D1212129974A42FF9740C3EFA
:10174B00FA7BFF120E7E7F541232B87BFF7A0A7936
:10175B00BA120E7E1231EB12330DD205E55924FF6E
:10176B009206122E67EF64027003021888BF040AF8
:10177B00052AE52AB40F03E4F52ABF080E152AC380
:10178B00E52A648094805003752A0EEF6401600390
:10179B000218627F541232B87BFF7A0A79CF120E8D
:1017AB007EE52AB40F0040030218359017BDF828C8
:1017BB0028730217EA0217EF0217F40217F9021740
:1017CB00FE02180302180802180D0218120218174D
:1017DB0002181C02182102182602182B02183012AC
:1017EB001E4D805B121EFF80561223D7805112278D
:1017FB00A9804C12282E8047121FA68042122B3133
:10180B00803D1222B18038122BAB8033122C2580F5
:10181B002E121ACD802912159980241224F5801FBF
:10182B00122E1B801A121BB980157F401232B87B07
:10183B00FF7A0A79DB120E7E7FE87E031200037DAE
:10184B00147F021230DC7F541232B87BFF7A0A7994
:10185B00ED120E7E1231EBE4FF1232B8AF2AEF33EA
:10186B0095E0FE7C007D1212129974A42FF9740C72
:10187B003EFA7BFF120E7E12330D0217657D147F2D
:04188B00041230DC37
:01188F002236
:10004E00E4F5237524FA75251E7526FFD200D2011C
:10005E00D202F587F5D0123332123337123327D24C
:10006E00BED297F563C2041218907E007F007D0504
:10007E007B007A007965121357D2B9C2CDD2AFD2B6
:10008E009CC298D2ACD203122D09E4FF1232B87B77
:10009E00FF7A0A79F9120E7E7F471232B87BFF7A09
:1000AE000B790E120E7E7F591232B87BFF7A0B79C6
:1000BE001B120E7ED2031232EF7FB87E0B1200039C
:1000CE0012328D7E007F067D007B007A00797412DD
:1000DE001357E4F527E4FDAF271232727F0A7E0034
:1000EE001200030527E527C3940240E9E4FD7FB023
:1000FE0012272240097BFF7A0B792B122FC1D208CF
:10010E007FC87E0012306E122F44C205C206122E18
:10011E0067EF6403703F7F401232B87BFF7A0B7932
:10012E003C120E7EE4F527D2087F647E0012306EFC
:10013E007F647E001200030527E527C3940A40E77B
:10014E00E4FBFAFD7FB01223467562017D147F0237
:10015E001230DC800512260E8F62E55575F00AA46A
:10016E0085F028F529E55BB403077DFFE4FF123225
:10017E0072E52660041526800B7526FFE4F525C270
:10018E0003122D09E4FF1232B8AF5BEF3395E0FE98
:10019E007C007D0912129974B22FF9740D3E753FD1
:1001AE00FFF54089417BFF7A0B794A7542008562E3
:1001BE0043754400855445120E7E20130320943758
:1001CE00D2031232EF7524FAC205C206122E678FC1
:1001DE0023BF030ED297D2087F0A7E0012306E1212
:1001EE00319AE523B40113D297D2087F0A7E00120A
:1001FE00306E12172B8003E4F523E4F527E52775FF
:10020E00F003A42474FFC3740495272465F8E6FB59
:10021E007D03123256E52775F003A42474F9E4FA2F
:10022E00FB786A7C00FDFE7F031212487F6A7D0315
:10023E00122FFB786BE6FF74152527F8A607052706
:10024E00E527C3940240B6E5256004152580287F76
:10025E005A1232B8E56375F00FA424DFF9740D3528
:10026E00F0753FFFF54089417BFF7A0779A3120EA7
:10027E007E75251EE4F563E4FF1230A67813A607FB
:10028E007F011230A67814A607E55B602724FC6078
:10029E00630470707F401232B8AE28AF297C007DA7
:1002AE000A1212AB8E3F8F407BFF7A0B795C120ED7
:1002BE007E0203527F401232B87813E6FF7E007C36
:1002CE00007D641212997DFF1212ABAA06AB07785D
:1002DE0014E6FF7E007C007D641212997DFF1212DF
:1002EE00AB8E418F428A3F8B407BFF7A0B79711226
:1002FE000E7E80507F401232B87BFF7A0B798A12C5
:10030E000E7E80407F401232B8AF697E007C007D49
:10031E00641212997DFF1212ABAA06AB07AF687E6C
:10032E00007C007D641212997DFF1212AB8E438FFA
:10033E00448A418B427BFF7A0B799A855E3F855FBB
:10034E0040120E7EE55B14700302048714700302E4
:10035E0005341470030205BD14700302070D240446
:10036E00600302071D7813E6FFD3943F4013EF940A
:10037E0066500E08E6FF943F4007EF94665002C2A7
:10038E000030160302071DE52324F8601724FC60D5
:10039E002224087029E56204FF7D017C001213E619
:1003AE008F62801AE56214FF7D017C001213E68FC6
:1003BE0062800B7D017C007F011213E68F6230009C
:1003CE000302071D7813E6C39434501508E6943FD4
:1003DE00400FE56204FF7D017C001213E68F62D2AE
:1003EE00007813E6D3943F401508E69434500FE599
:1003FE006214FF7D017C001213E68F62D200781327
:10040E00E6C39434501408E6C39434500D7D017C39
:10041E00007F011213E68F62D2007813E6D394B4F4
:10042E00401508E69466500FE56204FF7D017C00DE
:10043E001213E68F62D2007813E6C3946650150845
:10044E00E694B4400FE56214FF7D017C001213E6C2
:10045E008F62D2007813E6D394B4500302071D08BE
:10046E00E6D394B4500302071D7D017C007F011278
:10047E0013E68F62D20002071D7815E6C3944C5026
:10048E000908E6C3944C5002C20130160302071D40
:10049E00E52324F8601624FC602024087026E5620B
:1004AE0004FFE4FDFC1213E68F628018E56214FF70
:1004BE00E4FDFC1213E68F62800AE4FDFC7F01125C
:1004CE0013E68F6230010302071D7815E6D394B34D
:1004DE00401408E6944C500EE56204FFE4FDFC1255
:1004EE0013E68F62D2017815E6C3944C501408E6D9
:1004FE0094B3400EE56214FFE4FDFC1213E68F6226
:10050E00D2017815E6D394B3500302071D08E6D343
:10051E0094B3500302071DE4FDFC7F011213E68F16
:10052E0062D20102071D7816E6C3944C5002C20136
:10053E0030160302071DE52324F8601624FC602004
:10054E0024087026E56204FFE4FDFC1213E68F62B8
:10055E008018E56214FFE4FDFC1213E68F62800A38
:10056E00E4FDFC7F011213E68F6230010302071DCA
:10057E007816E6D394B3500302071D18E6D39406FB
:10058E00500302071D752701E527900E0B93FF7888
:10059E0015E6D39F400AE52795545004052780E8B9
:1005AE00E4FDFCAF271213E68F62D20102071D3065
:1005BE00160302071DE52324F8601724FC6022248D
:1005CE00087029E56204FF7D017C001213E68F623C
:1005DE00801AE56214FF7D017C001213E68F6280A3
:1005EE000B7D017C007F011213E68F62E529452801
:1005FE006003020703E55C24FE602C14604D14605A
:10060E007A1470030206BF240460030206F6E56244
:10061E00655470030206F6E56204FF7D017C00124C
:10062E0013E68F620206F6E55A6010E56204FF7D5E
:10063E00017C001213E68F620206F6E56214FF7D5E
:10064E00017C001213E68F620206F630020FE5629D
:10065E0004FF7D017C001213E68F62800DE56214AB
:10066E00FF7D017C001213E68F62E562B55402C273
:10067E0002E56264017071D202806DE55A6010E588
:10068E00622402FF7D017C001213E68F628059E521
:10069E0062B4010D7D017C00E4FF1213E68F6280CF
:1006AE0047E56224FEFF7D017C001213E68F628017
:1006BE0037300210E5622402FF7D017C001213E642
:1006CE008F62800EE56224FEFF7D017C001213E630
:1006DE008F62E55424FEFFE562D39F4002C202E51D
:1006EE0062C394025002D202E55575F00AA485F059
:1006FE0028F529801AE5291529700215288010750C
:10070E006201E55A24FF9204E4FD7FB01229B6E59A
:10071E005B64036004E55B70097F0A7E00120003D0
:10072E00801BE4F527C3740295272465F8E6FDAF18
:10073E00271232720527E527C3940240E830163B94
:10074E0030FF38E5626401701D30120B7B05FAFD37
:10075E007FB01223468009E4FBFAFD7FB0122346D8
:10076E00301103121C9DC2163017097D64AF56124C
:10077E001D7792177D147F031230DCE5246004157B
:0D078E00248005C2031232EFC29702017FE2
:01079B00223B
:10000300E4FDEF4E6018EF1F70011E7C66EC600884
:0E0013001CEDF5F0A4FD80F5D2AED2BE80E467
:0100210022BC
:10316F00AD07AC06ED7803CEC313CE13D8F9FDAC83
:10317F00067802CEC313CE13D8F92DFDEE3CFCED2D
:0B318F004C6007ED1D70F81C80F5225D
:02004800002294
:10306E008E3F8F40300830D2ECC2EEE54025E0F5C1
:10307E0040E53F33F53FE540453F6017E5401540DD
:10308E007002153F7FF47E0112316FB2EBD2AED2D9
:08309E00BE80E3C2ECC2EB228C
:102046008E378F388C398D3AE5397056E53A1460FB
:102056002314603314603824037047753927753AA2
:1020660010E538AE377802CEC313CE13D8F9F5385B
:102076008E378045753913753A88E537C313F537BA
:10208600E53813F5388032753909753AC4802A75F2
:102096003903753AE8E53825E0F538E53733F5379D
:1020A6008017753901753AF4E538AE377802C333CF
:1020B600CE33CED8F9F5388E37D2ECC2EEE53845B8
:1020C600376017E538153870021537AF3AAE391252
:0F20D600316FB2EBD2AED2BE80E3C2ECC2EB22CE
:0433410000401454E0
:0D331A00D2EDD2EDC2ED7F147E0002316FC6
:102F86007552FF85E85343E80FC2ECC2EFD2EED28A
:102F9600ED7F287E0012316F30EB13E552600F157E
:102FA600527F147E0012316FD2AED2BE80EAC2EDDD
:0A2FB6008553E8E5526002D322C300
:012FC00022EE
:100026008F51C2EC122F8653E8F0E551C4540F5499
:100036000F42E812331A53E8F0E551540F42E80232
:02004600331A6B
:1032B8008F3CC2EC122F86C2EFC2EEE53C4480FF81
:0332C800020026DB
:1032A3008F12C2EC122F86C2EFC2EEE512444054D5
:0532B3007FFF02002670
:102D0900E4F5E83003087F14FE12000380077F0111
:102D19007E0012000375E80312331A7F057E001244
:102D29000003122D5E122D5E75E80212331A7F011F
:102D39007E001200037F281200267F0C1200267FD6
:102D4900061200267F011200267F021200267F024A
:102D59007E0002000375E80312331A7F017E000228
:022D6900000365
:10328D007F011200267F027E001200037F021200D2
:06329D0026E4FF0232B836
:0E32FF008F50D2EFC2EE120026C2EFAF502267
:1030DC008F3A8D3B1230F9E53B600D153B7F20128A
:1030EC0032FFD2AED2BE80EFAF3A0230F9EF339559
:1030FC00E0FE74402FF58274333EF583E493FF02B7
:02310C0032B8D7
:1032EF00300304C2968002D2967F017E0002000353
:10325600ED14FEEED39400400EEF2E14F8E6FDEFCB
:0B3266002EF8A6051E80ECA807A603AA
:01327100223A
:02321200A8070B
:10321400E4F510F511FFEFC39D500EE62511F511ED
:10322400E43510F5100F0880EDED7C00AE10AF1101
:0332340012130072
:013237002274
:102FFB00ED14FEC3EE64809480402E7D01D3EE640D
:10300B0080F8ED648098501EEF2DF8E6FCE814F87C
:10301B00E6FBD39C400DA903EF2D14F8A604EF2D6E
:09302B00F8A6010D80D71E80CA31
:013034002279
:0300000002258254
:0C258200787FE4F6D8FD7581790225C948
:10117800E709F608DFFA8046E709F208DFFA803E59
:1011880088828C83E709F0A3DFFA8032E309F60846
:10119800DFFA8078E309F208DFFA807088828C83AE
:1011A800E309F0A3DFFA806489828A83E0A3F60862
:1011B800DFFA805889828A83E0A3F208DFFA804C3C
:1011C80080D280FA80C680D4806980F28033801013
:1011D80080A680EA809A80A880DA80E280CA80337C
:1011E80089828A83ECFAE493A3C8C582C8CCC583F4
:1011F800CCF0A3C8C582C8CCC583CCDFE9DEE780C4
:101208000D89828A83E493A3F608DFF9ECFAA9F042
:10121800EDFB2289828A83ECFAE0A3C8C582C8CC98
:10122800C583CCF0A3C8C582C8CCC583CCDFEADEB1
:10123800E880DB89828A83E493A3F208DFF980CC13
:1012480088F0EF60010E4E60C388F0ED2402B4040C
:101258000050B9F582EB2402B4040050AF232345B3
:0612680082239011C873FF
:10126E00BB010689828A83E0225002E722BBFE027E
:09127E00E32289828A83E49322B1
:10128700BB010689828A83F0225002F722BBFE0146
:02129700F32240
:10129900EF8DF0A4A8F0CF8CF0A428CE8DF0A42E69
:0212A900FE2223
:1012AB00BC000BBE0029EF8DF084FFADF022E4CC27
:1012BB00F875F008EF2FFFEE33FEEC33FCEE9DECF0
:1012CB00984005FCEE9DFE0FD5F0E9E4CEFD22ED36
:1012DB00F8F5F0EE8420D21CFEADF075F008EF2F80
:1012EB00FFED33FD4007985006D5F0F222C398FD71
:0512FB000FD5F0EA220E
:10130000C2D5EC30E709B2D5E4C39DFDE49CFCEE08
:1013100030E715B2D5E4C39FFFE49EFE1212ABC3C3
:10132000E49DFDE49CFC80031212AB30D507C3E4BE
:061330009FFFE49EFE2277
:10133600EB9FF5F0EA9E42F0E99D42F0E89C45F00D
:011346002284
:10134700E493FC740193FD740293FE740393FF22EC
:100E1C00E54B243FF8E6054B22783C300F02783F37
:100E2C00E475F0011213B002126E2008EB7F2ED283
:100E3C00088018EF540F2490D43440D4FF300C0B9E
:100E4C00EF24BFB41A0050032461FFE54C60021577
:100E5C004C054FE54F7002054E300F0D783CE47594
:100E6C00F0011213B0EF0212870232FF7403D20F9B
:100E7C008003E4C20FF54B8B3C8A3D893EE4F54C74
:100E8C00F54EF54FE54C60077F20120E5780F57537
:100E9C004DFFC209C208C20AC20BC20DC20EC2105B
:100EAC00120E25FF700D300F057F00120E68AF4F2C
:100EBC00AE4E22B4255FC2D5C20C120E25FF24D033
:100ECC00B40A00501A75F00A784C30D50508B6FFF4
:100EDC000106C6A426F620D5047002D20B80D924B4
:100EEC00CFB41A00EF5004C2E5D20C021068D2093C
:100EFC0080C6D20880C0D20A80BCD2D580BAD20DAE
:100F0C0080B47F20120E57200A077401B54C0040A4
:100F1C00F1120E1CFF120E57020E90D210D20E8040
:100F2C0095120E1CFB120E1CFA120E1CF94A4B7079
:100F3C000679397A117BFF200A2EE54C602A7E0057
:100F4C008E8275830012138360060EEE654D70F071
:100F5C00C2D5EBC0E0EAC0E0E9C0E0EE1210AFD0C1
:100F6C00E0F9D0E0FAD0E0FB12126EFF60AAEBC001
:100F7C00E0EAC0E0E9C0E0120E57D0E02401F9D05D
:100F8C00E03400FAD0E0FBE54D0460DCD54DD980AF
:100F9C00877BFF7A1079ABD20A809C79108002791A
:100FAC0008C20EC2108008D2D5790A8004790AC210
:100FBC00D5E54D047002F54DE4FAFDFEFF120E1C52
:100FCC00FC7B08200913120E1CFD7B1030080A1242
:100FDC000E1CFE120E1CFF7B20EC3382D592D550DA
:100FEC0013C3E43008069FFFE49EFEE42009039D32
:100FFC00FDE49CFCE4CBF8C209EC700CCFCECDCC5C
:10100C00E824F8F870F38017C3EF33FFEE33FEEDEE
:10101C0033FDEC33FCEB33FB994002FB0FD8E9EBCF
:10102C00300905F8D0E0C448B209C0E00AEC4D4ED6
:10103C004F78207B0070C2EAB54D0040BCC0E01276
:10104C0010B1D0F0D0E0200904C4C0E0C4B209C093
:10105C00F0120E40D0F0D5F0EB020E901213C00F30
:10106C002D530FA7580EFE4C0EFA420FAB4F0FB379
:10107C00440FB3490F13430FB9550F9D460F9D45B0
:10108C000F9D471159500F022D0F062E0F292B0FB4
:10109C000A230F272011472A0EC24800000F213FB8
:1010AC003F3F00790AA2D5200B14300D09B910026C
:1010BC000404B9080104A2D5200E02500104200A30
:0510CC0068920AB54C1A
:1010D100005034C0E07F20300B197F30A20A720E1D
:1010E100720D500F121108C20AC20EC20DC2107F3A
:1010F10030800F300D03E9C0E0120E57300D03D0E0
:10110100E0F9D0E0B54CCC300D177F30B9100C129E
:101111000E577F58300C077F788003B90803120EF1
:1011210057300A057F2D020E577F202010F87F2BA4
:10113100200EF322920A80CF286E756C6C29002D47
:1011410050434958D209120E1C3009F8C209784C93
:1011510030D50108F6020EC2120E1C2403B405009C
:101161004001E490114093120E48743A120E48D295
:071171000B754C04020FA7EF
:1032DD00C3EE6480948040028007C3E49FFFE49EA8
:0232ED00FE22BF
:10135700EF4E6012EF60010EEDBB010B89828A83AD
:10136700F0A3DFFCDEFA2289F05007F709DFFCA9BA
:0C137700F022BBFEFCF309DFFCA9F02211
:10258E0002004EE493A3F8E493A34003F68001F215
:10259E0008DFF48029E493A3F85407240CC8C3334E
:1025AE00C4540F4420C8834004F456800146F6DF1D
:1025BE00E4800B01020408102040809032CBE47EB0
:1025CE00019360BCA3FF543F30E509541FFEE49312
:1025DE00A360010ECF54C025E060A840B8E493A3D9
:1025EE00FAE493A3F8E493A3C8C582C8CAC583CA04
:1025FE00F0A3C8C582C8CAC583CADFE9DEE780BEBC
:0132DC0000F1
:10138300BB010CE58229F582E5833AF583E022501F
:1013930006E92582F8E622BBFE06E92582F8E22269
:0D13A300E58229F582E5833AF583E4932283
:1013B000FAE6FB0808E6F925F0F618E6CA3AF6223E
:1013C000D083D082F8E4937012740193700DA3A3BC
:1013D00093F8740193F5828883E4737402936860D0
:0613E000EFA3A3A380DFD0
:00000001FF
